:1000000009C021C020C01FC01EC01DC01CC01BC015
:100010001AC019C011241FBECFE9CDBF10E0A0E661
:10002000B0E0E6EFF2E003C0C89531960D92A0363D
:10003000B107D1F710E0A0E6B0E001C01D92A036F4
:10004000B107E1F701C0DCCFCFE9D0E0DEBFCDBF23
:1000500083E287B981E886B988E084BB80E187BB09
:10006000369A3699FECF369A3699FECF25B1822F31
:100070008D196AE027D1D80E3327442737FD4095E4
:10008000542F952F842F732F622F39D0E62EF72E01
:10009000082F192F6D2D7727882777FD8095982FAA
:1000A0002ED026E636E646EA5FE3A0D0262F372F8D
:1000B000482F592F912F802F7F2D6E2D2DD0181660
:1000C0001CF020E030E00DC080E188BB80E090E0D3
:1000D000000000000000019684369105C9F724E66F
:1000E00030E018BA84E690E004C000000000000090
:1000F000019728173907CCF3B6CFE89403C097FBD4
:100100000EF4D5D0B62F672F782F892F9EE90024C3
:1001100027C00ED05EF004C00BD026F001C008D07E
:1001200019F020F48FEF089580E0089581E008959C
:1001300097FB092E052600F868942DD0E89407FC5B
:1001400007C0621773078407950721F008F400942D
:100150000794989408959A95BB0F661F771F881F80
:1001600011249923A1F08823B2F79F3F59F0BB0FC8
:1001700048F421F4002011F460FF04C06F5F7F4F4A
:100180008F4F9F4F881F9795879597F9089529C09E
:10019000052E092607FA440F551F5F3F79F0AA275D
:1001A000A51708F051E04795880F991F9F3F31F040
:1001B000BB27B91708F091E0879508959F919F910B
:1001C00011247DC097FB880F991F9F3F31F0BB27FB
:1001D000B91708F091E0879508959F919F91112498
:1001E0006EC066277727882799270895D1DF01D029
:1001F000B7CF992339F0552329F09F575F57950FB3
:1002000013F4CAF1F1CF91589F3FE1F3A62F0024D8
:100210001124BB2766275527F8E0A69520F4020E87
:10022000131EB41F651F220F331F441F551FFA955D
:10023000A1F7F8E0E72F7727F8E0E69520F4130E12
:10024000B41F651F7A1F330F441F551FAA1FFA954D
:10025000A1F7F82F8827F69520F4B40F651F7A1FB1
:100260008E1F440F551FAA1FEE1FFF23A1F78823DF
:100270001AF4939539F423C0000C111CBB1F661FA0
:10028000771F881F0128089597FB8EDF9F3738F06E
:10029000FEE9F91B982F872F762F6B2F05C0A1CF72
:1002A0009695879577956795F150D0F73EF49095A0
:1002B0008095709561957F4F8F4F9F4F08959FEF69
:1002C00080EC089587FB082E062687FD819567FD43
:1002D000619505D00EF4919507FC81950895991BC1
:1002E00079E004C0991F961708F0961B881F7A952D
:0602F000C9F78095089596
:00000001FF
